:107C000001C002C1112484B7882361F0982F9A70B3
:107C1000923041F081FF02C097EF94BF282E80E0A0
:107C2000DED0EEC185E08093810082E08093C000C9
:107C300088E18093C10086E08093C20080E1809358
:107C4000C4008EE0CCD0259A86E020E33CEF91E0A2
:107C5000309385002093840096BBB09BFECF1D9A85
:107C6000A8954091C00047FD02C0815089F723E0EC
:107C7000D22ECC24C39435E0B32E41E1A42EA3D060
:107C8000813471F4A0D0182FB0D081E0123821F0E7
:107C900088E0113809F083E08FD080E18DD0EFCFFC
:107CA000823419F484E1A9D0F8CF853411F485E049
:107CB000FACF853541F487D0C82F85D0D82FCC0F87
:107CC000DD1F93D0EACF863521F484E096D080E0A2
:107CD000E3CF843609F045C076D075D0182F73D025
:107CE000082F812C9924939474018FEFE81AF80AD5
:107CF0006AD0F401808347011E11F6CF76D0053497
:107D000091F4E12EF12C10E000E0F801F3950E154E
:107D10001F0509F4C2CF6081C8018C0F9D1F8CD054
:107D20000F5F1F4FF2CFFE01D7BEE89507B600FCEC
:107D3000FDCFFE01A0E0B1E0CD0102962D913C9176
:107D40000901C7BEE89511243296DC011813F4CF5F
:107D5000FE01B7BEE89507B600FCFDCFA7BEE895CB
:107D60009CCF8437D1F42FD02ED0182F2CD0082FB1
:107D70003CD07E01053451F4C70156D01DD01150BE
:107D8000FFEFEF1AFF0A1111F7CF87CFF7018591A7
:107D90007F0112D01150D1F780CF853739F425D02B
:107DA0008EE10AD085E908D08FE076CF813509F0E1
:107DB00088CF88E014D085CF9091C00095FFFCCF8C
:107DC0008093C60008958091C00087FFFCCF80910A
:107DD000C00084FD01C0A8958091C6000895E0E62A
:107DE000F0E098E1908380830895EDDF803219F010
:107DF00088E0F5DFFFCF84E1DFCFCF93C82FE3DF4B
:107E0000C150E9F7CF91F1CFFC010A0167BFE895B6
:107E1000112407B600FCFDCF667029F0452B19F43C
:107E200081E187BFE8950895F999FECF92BD81BDA4
:107E3000F89A992780B50895262FF999FECF1FBA91
:107E400092BD81BD20BD0FB6F894FA9AF99A0FBE83
:107E50000196089556657273696F6E3D382E310034
:107E60004F505449424F4F545F435553544F4D5612
:107E700045523D30004465766963653D61746D65CA
:107E800067613332387000465F4350553D313630BC
:107E900030303030304C00424947424F4F543D3132
:107EA000004275696C743A4A756C20203720323074
:107EB00032303A31313A33333A3334005541525447
:107EC0003D3000424155445F524154453D313135CA
:107ED00032303000535550504F52545F4545505248
:107EE0004F4D3D31004C45443D4235004C45445FCB
:107EF00053544152545F464C41534845533D33001F
:027FFE00010878
:0400000300007C007D
:00000001FF
